:100000000C946A000C9400000C9400000C94000006
:100010000C9400000C9400000C9400000C94000060
:100020000C9400000C9400000C9400000C94000050
:100030000C9400000C9400000C9400000C94000040
:100040000C94CC000C9400000C9499000C940000CB
:100050000C9400000C9400000C9400000C94000020
:100060000C9400000C9400001027E80364000A00C0
:1000700001000010000110000100000000000A0053
:100080000000000000000000000000000000000070
:100090000000000000000000000000000000000060
:1000A0000000000000000000000000000000000050
:1000B0000A0A0A0A0A0A0A0A0A0A0A0A0A0A0A0AA0
:1000C000020002007A00020004007C000100080324
:1000D0007E000000F894EE27EFBBF1E0F5BFE5BF2E
:1000E0008DE0A2E0BB27ED938A95E9F780E098E0E8
:1000F000A0E0B1E0ED930197E9F7E0ECF0E0859145
:100100009591009761F0A591B59105901590BF016B
:10011000F00105900D920197E1F7FB01F0CFE8E0C7
:10012000EEBBEFEFEDBFE8E0EEBFC0E0D3E00C9434
:10013000A203AA93EA93FA93EFB7EA931A930A9366
:100140001091C0000091C600E12FEC71E9F4E0913C
:10015000F303EF5FE093F303E150F0E0E652FC4F6E
:100160000083A091F303A93119F4E0E0E093F303D5
:10017000A091F503AF5FA093F503A93129F4E0E066
:10018000E093F503689437F809911991E991EFBF6D
:10019000F991E991A99118950A921A926A937A9322
:1001A0008A939A93AA93BA93EA93FA93EFB7EA934E
:1001B000E0913A03F0913B033196E0933A03F093D8
:1001C0003B030E94AE21E1E5F1E00E94E82B0E2EF8
:1001D0000E94AE21E3EAF2E00E94E82BE02909F454
:1001E00016C2A0913803B0913903E4E1F0E00E9417
:1001F000FA2B0E2EE0910503F0E074970E94EE2B8F
:100200000E22A0911F03EEE00E94DE2BE02121F0E0
:10021000E0911F03EF5F03C025FC03C0E0E0E09323
:100220001F03A0911F03AE3011F4689425F8E091EC
:100230003803E0930503A0912803A13029F4F79B2C
:1002400002C0F79801C0F79AE1E02E260E94B32180
:100250000E94BC21E093BE03F093BF036093C003F0
:100260007093C1030E94C321A2EAB3E00E94C82197
:100270000E94CF21AEECB3E00E94C8210E94D4219D
:100280000E94DD210E94142BE093A203F093A303AC
:100290006093A4037093A503A091CE03B091CF0304
:1002A0008091D0039091D103E0E0F0E060E772E448
:1002B0000E94142BE093CE03F093CF036093D003FE
:1002C0007093D1030E94E2210E94E7210E2E0E942A
:1002D000EC210E94E721E02161F1E091CE03F09151
:1002E000CF036091D0037091D1030E94D4210E946A
:1002F000142BE093CA03F093CB036093CC03709369
:10030000CD030E94F121ACE4B3E00E94FA21A09158
:10031000CA03B091CB038091CC039091CD030E948E
:10032000BC21E093AA03F093AB036093AC037093FA
:10033000AD030E94FF210E9410220E94762AE093C2
:10034000B203F093B3036093B4037093B5030E94B8
:10035000FF210E9419220E94762AE093D603F0938F
:10036000D7036093D8037093D9030E9422220E947E
:100370002B220E943E22AAE8B3E00E94052A0E9496
:10038000DC2C0E942222AAE0B0E080E090E00E94F3
:10039000202C0E9419220E943A2A0E94592B70F0A8
:1003A000E0E0E093D603E093D703E093D803E09333
:1003B000D9030E94432231960E944822E0918E0385
:1003C000F0918F036091900370919103A091B60317
:1003D000B091B7038091B8039091B9030E94C62AE7
:1003E000DF01CB010E94BC21E093C203F093C30361
:1003F0006093C4037093C5030E944D220E94762A25
:100400000E945622E0910F03F0E00E945F220E94BA
:10041000BB2B0E946822ACE6B3E00E9477220E94C8
:10042000B3210E943C2D3CF5A091C203B091C303BF
:100430008091C4039091C5030E947C227F936F93A7
:10044000FF93EF93A091BE03B091BF038091C003CF
:100450009091C1030E947C22AF91BF918F919F9197
:100460000E94142BE093BA03F093BB036093BC0388
:100470007093BD0309C0E0E0E093BA03E093BB03CF
:10048000E093BC03E093BD03A091BD03AA238AF4CB
:100490000E9483220E948C2218F40E94932208C09A
:1004A0000E949A220E94D029A4E7B3E00E947722FA
:1004B00014C00E948322E0E0F0EC69E774E40E943B
:1004C000592B09F008F403C00E94932206C00E9431
:1004D0009A22A4E7B3E00E9477220E94A3220E94FE
:1004E000AC220E94762A0E94B522E091A203F091EC
:1004F000A3036091A4037091A5030E94BE220E94F1
:10050000592B68F5E091AA03F091AB036091AC031D
:100510007091AD030E94BE220E94762AE093A6034A
:10052000F093A7036093A8037093A9030E94BE22CF
:100530000E94C7220E946F2ADF01CB010E94F12195
:100540000E94142BA0E0B0E081E695E40E94C62A48
:10055000A8E6B3E00E947722689424F802C0E0E1A4
:100560002E260E94A3220E94D0220E94762AE09387
:10057000AE03F093AF036093B0037093B1030E9496
:10058000D022E0E0F0E060E87FE30E94592B09F020
:1005900008F412C0E093AE03E093AF03E093B0031E
:1005A000E093B1030E94D922EF5FFF4F6F4F7F4F5F
:1005B0000E94E2220E94EB220E94F122A034E2E497
:1005C000BE07EFE08E07E0E09E0778F0E0E0E09302
:1005D0005A03E0935B03E0935C03E0935D03AEE3B7
:1005E000B0E00E94FA220E94112D0E94AC220E94CB
:1005F000FF22ACE3B3E00E94FA21A0911D03AC33CB
:1006000008F4F298A0911D03AC3309F4F29A0E9409
:10061000AE21A33AE2E0BE0709F06BC0A0911C0333
:100620000E9403230E9408230E94FA220E94002CA9
:100630000E941123E02191F0E0911D03EF5FE09310
:100640001D03E0911C03F0E03296A0911D03B0E081
:10065000EA17FB0719F4ECE3E0931D03E0E0E093F5
:100660003A03E0933B03D394A0911003A13028F404
:10067000E0911003EF5FE09310030E941823E8E578
:10068000F2E00E94F42B0E2E0E941D23E021E9F0DF
:10069000E0915003F09151033196E0935003F093B1
:1006A00051030E9418230E942223EA1BFB0BE093B4
:1006B0005603F09357030E9408230E943C2D2CF40C
:1006C000E0E0E0935003E0935103ECE3ED1589F48F
:1006D000DD24C394EC1569F4CC24E0910003EF5FB2
:1006E000E0930003A0910003A43119F4E0E0E0934B
:1006F0000003E991EFBFF991E991B991A99199911D
:10070000899179916991199009901895AA93E88136
:10071000E066E0937C0085E28A95F1F7E0917A004B
:10072000E064E0937A00E0917A00E071E1F3E09117
:100730007A00E061E0937A00E0917800F09179002E
:1007400021960895EF97279780E4A6E0B0E0E0E8CF
:10075000F0E00E94512DFF2401E021E0E0E8E09369
:100760006100E0E0E0936100EFE0E4B9E1E0E5B9C9
:10077000E0E0E7B9E4E0E8B9EAEFEAB9E7EEEBB9BF
:10078000E0E0E4BDE3E0E5BDE0E0E6BDE7BDE8BDF7
:10079000E1EAE0938000E2E0E0938100E0E0E093B2
:1007A0008500E0938400E0938700E0938600E09367
:1007B0008900E0938800E0938B00E0938A00E09347
:1007C000B600E1EAE093B000E2E0E093B100E0E0DF
:1007D000E093B200E093B300E093B400E1E0E09373
:1007E0006E00E0E0E0936F00E0937000E09369003A
:1007F000EDBBE0936800E093C000E8E9E093C1003E
:10080000E6E0E093C200E0E0E093C500E7E4E093B7
:10081000C400E0E8E0BFE0E0E0937F00E0937E000A
:10082000E0E6E0937C00E6E2E0937A00E0E0E0932B
:100830007B00ECBDE093BC0078945F9A0E94272374
:100840000E942B230E9438230E9445230E942723C5
:10085000EAE06E1668F4ACE2B0E00E945223A8E22F
:10086000B0E0E0E00E94212DA9E2B0E00E94212D3D
:10087000EAE09E1650F4A2E3B0E00E945223AAE3FD
:10088000B0E00E945223689426F8EAE0BE1618F4FD
:10089000689430F827F8689433F8E4E1E0931103A2
:1008A0000E9457230E945E230E946523E8ECF0E03B
:1008B000E0936203F0936303A0E0B0E00E94052D93
:1008C000E0931203A1E0B0E00E94052DE093130332
:1008D000A2E0B0E00E94052DE0931403A3E0B0E095
:1008E0000E94052DE0931603A4E0B0E00E94052DC0
:1008F000EC8FA5E0B0E00E94052DED8FA6E0B0E002
:100900000E94052DEE8FA7E0B0E00E94052DE09338
:100910001703A8E0B0E00E94052DE0931803A9E0BA
:10092000B0E00E94052DE0931903F798F198AAE032
:10093000B0E00E94052DE0931C03AAE2B0E00E9403
:10094000012D0E946C23A4E1B0E00E94052DE88FE8
:10095000A5E1B0E00E94052DE98FA6E1B0E00E947C
:10096000052DEA8FABE0B0E00E94052DEC8BACE0EA
:10097000B0E00E94052DED8BADE0B0E00E94052DAA
:10098000EE8BAEE2B0E00E94012DEB87FC87AEE07B
:10099000B0E00E94052DE0932903AFE0B0E00E9493
:1009A000052DE0932B03A0E1B0E00E94052DE0931C
:1009B0002A03AEE3B0E00E94FD2C0E94E222ACE2EA
:1009C000B0E00E94012DAEE9B3E00E9471230E94C5
:1009D000C722ACE3B3E00E94FA210E94AC220E943D
:1009E00078230E94B522A1E1B0E00E94052D3E2FA0
:1009F000A0E3B0E00E94012DEF87F88BA2E1B0E008
:100A00000E94052DE8A3A3E1B0E00E94052DEF8F21
:100A1000A2E3B0E00E94012DA2EBB3E00E9471239B
:100A2000AAE3B0E00E94012DA2EDB3E00E94712381
:100A30000E944D220E9478230E945622A4E3B0E037
:100A40000E94012D0E947C23A8E3B0E00E94012DAA
:100A50000E94BB2B0E948123A7E1B0E00E94052DDC
:100A60000E944C2D23F8A6E3B0E00E94012D0E94C5
:100A70008A23A8E1B0E00E94052DE0930703A9E1D5
:100A8000B0E00E94052DE0930903AAE1B0E00E94C6
:100A9000052DE0930A03ABE1B0E00E94052DE09341
:100AA0000B03ACE1B0E00E94052DE0930C03ADE137
:100AB000B0E00E94052DE0930D03AEE1B0E00E948E
:100AC000052DE0932003AFE1B0E00E94052DE093F7
:100AD0002103A0E2B0E00E94052DE0932203A1E2F1
:100AE000B0E00E94052DE0932303A2E2B0E00E9453
:100AF000052DE0932403A3E2B0E00E94052DE093CE
:100B00002503A4E2B0E00E94052DE0932603A5E2B0
:100B1000B0E00E94052DE0932703ACE3B0E00E9413
:100B2000012D0E944822A6E2B0E00E94052DE0932C
:100B30000F03A7E2B0E00E94052D0E944C2D36F86D
:100B400036FE0BC0A8E2B0E00E94052DCE2EA9E231
:100B5000B0E00E94052DE0930003A0910203A431B0
:100B600028F4E0910203EF5FE0930203A0910203F7
:100B7000A431A1F4E0E0E0932D03E0932E03EBE039
:100B8000F0E0E0935403F0935503E8EBE0932F0378
:100B9000E0E0E093F303EAE0E0930203A091F303C3
:100BA000AB30C1F4E091DD03E0932D03E091DE036F
:100BB000E0932E03E091DF03F0E0E0935403F09321
:100BC0005503E091E003E0932F03E0E0E093F303AB
:100BD000E0930203A091F303AC30C0F0E0E0E093B7
:100BE000DA03E093DB03E093DC03E093DD03E093BF
:100BF000DE030E945723E0E0E093E103E093E20389
:100C0000E093E303E093E403E093F303E8EC5E1680
:100C100030F45394E4E1E51511F4E1E04E2E0E9426
:100C20008F23A6E00E949723EF83F887E7E2E09303
:100C30007A000E948F23A0E00E949E233B97C8F178
:100C4000A0E00E949723662777270E94A323A8EE9F
:100C5000B3E080E090E00E944B2CDF01CB010E94CA
:100C6000AC23662777270E948D2C0E94A323AEE831
:100C7000B3E00E943C2A0E94DC2CE0910803EF5F65
:100C8000E0930803E0910703A0910803AE1778F002
:100C90000E94B123E0938603F09387036093880357
:100CA0007093890323FC03C0E0E0E0930803E89419
:100CB000F3F80E94BA230E942B230E94C123A2E0D2
:100CC0000E949723DF01E5E0F0E00E94502C8E2E79
:100CD0000E94BA230E9445238AE48A95F1F70E9474
:100CE00038230E94C123A7E00E949E230E94C823AC
:100CF0000E94BA23E7EAE0937A00A5E00E949E23CF
:100D00001E2F0E94BA23E7EAE0937A00A0E00E9437
:100D10009E23AE2E0E94BA23E1E0E51591F50E94D4
:100D2000CD23E2E3F0E00E94FA2B0E2E0E94D223A4
:100D30000E94F42BE02111F0E5E0EA8BA12FE2E321
:100D40000E94E32B0E2EEAEF0E94DE2BE02111F031
:100D5000E6E0EA8B0E94D2230E94FA2B0E2E0E941C
:100D6000D623E02911F0E7E0EA8BA12FEAEF0E94F9
:100D7000E32B0E2EEEE10E94DE2BE02911F0E8E0DD
:100D8000EA8B0E94D2230E94FA2B0E94DC2339F0C6
:100D9000E1E0EA8BE8E2F0E00E94C82307C00E948D
:100DA000D6230E94DC2311F0E2E0EA8BA12FEAEFC8
:100DB0000E94E32B0E94DC2311F0E3E008C0A12F86
:100DC000EEE10E94DE2B0E94DC2319F0E4E0EA8BC6
:100DD0001CE30E94E8230E94CA2B0E94F0230E9479
:100DE000CA2BE021E1290E2EAA89E1E00E94C52B41
:100DF0000E2AE2E00E94C52BE02929F0E12FF0E065
:100E00000E94C82318E20E94E8230E94C52B0E947A
:100E1000F0230E94C52BE021E12911F00E94FA2362
:100E2000AA890E940024AA89E8E00E94C52BE02933
:100E300009F018E20E9405240E940B240E94DE2B78
:100E4000E021D1F06894F3F8013021F4F398F49A9A
:100E500002E012C0023059F4F498F59AAE8DA13038
:100E600010F003E003C0F598F39A01E005C00330E9
:100E700019F4F598F39A01E00E94CD23D39708F472
:100E800057C00E9415240E941A24E02F0E9421249A
:100E900020F0E8ECF0E00E94C823E02F0E9431240B
:100EA0000E944124AC91A13008F441C00E94482422
:100EB0000E9451240E94472D4CF40E9441240E941C
:100EC0005D240E94852B0E94682423C00E94712407
:100ED0000E947324EF930E9471240E947C24AF919E
:100EE000EA2379F00E9441240E945D240E948A2B0B
:100EF000A0937603B093770380937803909379035C
:100F000008C00E9471240E9485241CF00E948F2436
:100F10000EC0A0917603B0917703809178039091F1
:100F200079030E949E240E948D2C0E94C82304C035
:100F30000E94FA230E948F240E94A3240E94A924C5
:100F40000E220E94AE24E02139F0E0913403E093B8
:100F50001E036894F0F821F80E941524309721F4BC
:100F6000E0E0E0931F0306C0A0911F03A23010F43D
:100F7000E89425F80E941524E0933803F093390390
:100F80000E941524309719F4E89421F815C0A0E0C8
:100F900021FCA1E0E0E00E94C52B0E2EA0911E03D3
:100FA000E0E00E94E32BE02139F0E0E0E0931E0353
:100FB0000E94FA23E89422F8E09104030E94CD23D2
:100FC000F0E0AE17BF0720F0E0913403E093040394
:100FD000E0910403F0E035970E94CD23AE17BF07E0
:100FE000B0F4E0913403E0930403A0E025FCA1E019
:100FF000E1E00E94C52B0E2E0E94B52441F0E2E0F4
:10100000E0932C03E89425F8E0E0E0931F03A0911F
:101010001E03A13080F0689422F80E941524A0914C
:101020001E03B0E0AE17BF0728F0E0911E03F0E00A
:101030000E94C82302C0E89422F80E94BD240E94A6
:10104000C0240E94102C0E22A09129030E94C724C4
:101050001E2E0E94BD240E94C0240E94082C0E2235
:10106000A0912A030E94C7241E2A0E94BD24A12FFA
:10107000E2E30E94E32BE021E12979F00E94FA23C8
:10108000A0912C03A13021F4EAE0F0E00E94C823F3
:10109000E0912C03E150E0932C030E94CC240E221B
:1010A000A0E031FCA1E00E94C72431F0689431F83F
:1010B0000E9415240E94E2240E94CC24E02161F1C8
:1010C0000E94E7240E94EF24A4F0A0918203B09133
:1010D0008303EB85FC85EA1BFB0BA3E0B0E00E94D9
:1010E000462C0E94F724AE1BBF0BA0936403B09361
:1010F00065030E94E7240E943C2D2CF40E94FC24EE
:1011000032970E94E224A0916503AA232AF4E0E02A
:10111000E0936403E09365030E9401250E94422D41
:1011200074F50E9401250E948A2B0E94EF2474F01E
:10113000AB85BC85E0918203F0918303EA1BFB0B36
:101140000E94F724EA0FFB1F0E94E2240E9401255F
:101150000E948A2BA230E0E0BE07E0E08E07E0E0CC
:101160009E072CF00E94FC2431960E94E2240E94EB
:10117000F724A93CE0E0BE0714F00E945E230E9421
:10118000FC240E94CD23AE17BF0710F4E89431F879
:101190000E94FC240E94CD23EA17FB0720F40E9442
:1011A000FC240E94C8230E940E250E947F2B0E2E35
:1011B000A0E032FCA1E00E94C72441F0689432F81C
:1011C0000E941D25E0936603F09367030E940E259D
:1011D0000E94592B09F008F435C00E942225DF0136
:1011E000CB01E0E0F0E060E070E40E94592B09F0F0
:1011F00008F410C00E942225A0E0B0E080E890E44E
:101200000E94C62A0E9431250E943625A6E6B3E038
:101210000E9477220E9422250E94322D54F4E8A1D8
:10122000F0E00E943125AE1BBF0BA0936603B09384
:101230006703A0916703AA232AF4E0E0E093660322
:10124000E09367030E940E250E94592BC0F50E946F
:101250003B25DF01CB01E0E0F0E060E470E40E94B8
:10126000592B09F008F414C00E943B25A0E0B0E01F
:1012700080EA90E40E94C62ADF01CB010E94462545
:101280000E944B250E94762AA6E6B3E00E947722B0
:101290000E943B250E94322D54F4EF8DF0E00E9415
:1012A0003125EA0FFB1FE0936603F09367030E946A
:1012B0003125A13DE7E0BE0714F00E9465230E949E
:1012C0001D25DF010E944625AE17BF0710F4E894E4
:1012D00032F80E941D25DF010E944625EA17FB0710
:1012E00020F40E9431250E9450250E9455250E941D
:1012F000102C0E2EA0E034FCA1E00E94C72431F097
:10130000689434F80E941D250E945C250E94552592
:101310000E94422D5CF50E9461250E94EF249CF002
:10132000E0911303F0E0A0917E03B0917F03AE1B28
:10133000BF0BE3E0F0E00E946A25AE1BBF0BA09359
:101340006E03B0936F030E9461250E943C2D2CF424
:101350000E94712532970E945C25A0916F03AA23F9
:101360002AF4E0E0E0936E03E0936F030E945525BA
:101370000E94472D8CF50E947625A430E0E0BE0740
:10138000E0E08E07E0E09E078CF0A0911303BB27FE
:10139000E0917E03F0917F03AE1BBF0BE2E0F0E033
:1013A0000E946A25EA0FFB1F0E945C250E94762599
:1013B0000E943C2D2CF40E94712532960E945C25DF
:1013C000A0916E03B0916F03A13DE7E0BE0724F04A
:1013D000E0EDF7E00E945C250E941D25DF010E94E0
:1013E0007125AE17BF0710F4E89434F80E941D254C
:1013F000DF010E947125EA17FB0730F4A0916E030C
:10140000B0916F030E9450251333E0F0E0E0E093C9
:101410000603A0911E03A13018F0E2E0E0932C0334
:10142000E0E0E0931E03E12FF0E0F2970E944B25ED
:10143000A6EFB8E28CE99FE30E94C62A0E94032A25
:101440001E2F01C010E00E941524E987FA87A82DFD
:10145000E4E60E94DE2B6E2F0E2E0E9486250E22C1
:10146000AE81EDE50E94CA2B0E948D251E2E062E10
:101470000E9486250E220E94A924E0211E2A0E9495
:1014800022230E9418230E94E82B0E9494250E9488
:101490001D23E021E12931F1E0913C03F0913D036E
:1014A000ACE2B0E00E949C250E94A2250E944D2241
:1014B0000E94FF220E94AF250E94B425EC2DA8E2D5
:1014C000B0E00E94B825E0910003A9E2B0E00E94DC
:1014D000212D0E9427235F98A8EEB3E00E94C62921
:1014E0005F98FECFAB2D0E94BE250E94A924E0216B
:1014F00031F0E894F2F827F8E0E0E09333030E943B
:10150000C3250E94A924E02171F0E0913303EF5F2D
:10151000E0933303A0913303AA3029F4E0E0E09391
:101520003303E09328030E94C3250E94D0250E2296
:101530000E94A924E02171F06894F2F8E091280358
:10154000EF5FE0932803A0912803A33019F4E1E0B2
:10155000E0932803E0912803E03029F4E0E0E093F1
:10156000B400F7980FC0A0912803A13019F4E091BE
:10157000190306C0A0912803A23021F4F79AEFEFD7
:10158000E093B4000E94CD230E94E7210E2EA12FEC
:10159000E0E00E94E32B0E220E94B52401F1E091CD
:1015A0000303EF5FE0930303A0910303E5E00E94D0
:1015B000E32B0E2EE4E10E94DE2BE02141F0E091CE
:1015C0000303E170AFEFEA02F001E093B400A091F1
:1015D0000303A03118F0E0E0E093030326C0A0E08D
:1015E00030FCA1E0E1E00E94C52B0E2EA091280363
:1015F0000E94C724D1F0E0913203EF5FE093320301
:10160000A0913203A13019F4EFEFE093B400A09160
:101610003203A33019F4E0E0E093B400A091320368
:10162000A43019F4E0E0E0933203E0911803E09372
:10163000B300EAE0E91518F4E894F1F826F80E94FE
:10164000D725A0E026FCA1E00E94DD25A0E0F1FC6A
:10165000A1E00E94DD250E94A924E02139F16894CF
:10166000F1F8E0910E03EF5FE0930E03E0E0E98B09
:10167000A989A53088F40E94E225A081A13018F044
:10168000E5E0E98B05C0E0910E03EF5FE0930E0308
:10169000E989EF5FE98BECCFA0910E03A53018F03C
:1016A000E0E0E0930E030E94E22520810E94D7250E
:1016B000A0911B03EFEF0E94DE2BE02121F0E091CF
:1016C0001B03EF5F03C0E894F1F8E0E0E0931B0335
:1016D000A0911B03A43109F02EC1AE81E0E00E946D
:1016E000D92B0E2E0E94A924E02119F0EE81E150A1
:1016F000EE83233610F423E61EC121E0E0E0E09300
:101700000E03E0911203A0E0B0E00E94B825E09142
:101710001303A1E0B0E00E94B825E0911403A2E019
:10172000B0E00E94B825E0911603A3E0B0E00E946B
:10173000B825EC8DA4E0B0E00E94B825ED8DA5E0C1
:10174000B0E00E94B825EE8DA6E0B0E00E94B8257A
:10175000E0911703A7E0B0E00E94B825E0911803DC
:10176000A8E0B0E00E94B825E0911903A9E0B0E03C
:101770000E94B825E0911C03AAE0B0E00E94B825C1
:101780000E94AC23AAE2B0E00E949C25E88DA4E16F
:10179000B0E00E94B825E98DA5E1B0E00E94B8252F
:1017A000EA8DA6E1B0E00E94B825EC89ABE0B0E09C
:1017B0000E94B825ED89ACE0B0E00E94B825EE8922
:1017C000ADE0B0E00E94B825EB85FC85AEE2B0E06C
:1017D0000E949C25E0912903AEE0B0E00E94B8256C
:1017E000E0912B03AFE0B0E00E94B825E0912A031E
:1017F000A0E1B0E00E94B825E32FA1E1B0E00E9493
:10180000B825EF85F889A0E3B0E00E949C25E8A107
:10181000A2E1B0E00E94B825EF8DA3E1B0E00E9404
:10182000B8250E94A2250E94E825A4E3B0E00E940A
:101830009C25E0915E03F0915F03A8E3B0E00E9475
:101840009C25E0E023FCE1E0A7E1B0E00E94B825A0
:101850000E942223A6E3B0E00E949C25E0910703AA
:10186000A8E1B0E00E94B825E0910903A9E1B0E049
:101870000E94B825E0910A03AAE1B0E00E94B825D1
:10188000E0910B03ABE1B0E00E94B825E0910C03BE
:10189000ACE1B0E00E94B825E0910D03ADE1B0E00D
:1018A0000E94B8250E944D220E94FF220E94AF256F
:1018B000E0912003AEE1B0E00E94B825E091210361
:1018C000AFE1B0E00E94B825E0912203A0E2B0E0D1
:1018D0000E94B825E0912303A1E2B0E00E94B82560
:1018E000E0912403A2E2B0E00E94B825E091250334
:1018F000A3E2B0E00E94B825E0912603A4E2B0E0A4
:101900000E94B825E0912703A5E2B0E00E94B82527
:101910000E94B425E0910F03A6E2B0E00E94B82532
:10192000E0E036FCE1E0A7E2B0E00E94B8250E94CA
:10193000EB22E1E04E2E0E94D725A0E0F1FCA1E0D1
:101940000E94DD25AE81E4E60E94D42B0E948D2505
:1019500051F06894F1F8EE81EF5FEE83AE81A4362A
:1019600011F4E0E0EE83EAE0E61510F4E894F0F814
:101970000E94A3240E94AE240E22AE81E0E00E94C9
:10198000CF2B0E948D2551F06894F0F8EE81E15044
:10199000EE83AE81AF3F11F4E3E6EE830E940524AF
:1019A000A22FE3E60E94C52BE021C1F00E94ED25A5
:1019B000A9F4A0913003A43119F4E7E0E0933003D7
:1019C000E0E0E0933103E894F3F8A0913003A33012
:1019D00028F0E0913003E150E0933003AB2DEAE0D2
:1019E0000E94DE2B0E2EA22FE3E60E94C52BE021E3
:1019F000C1F00E94ED25A9F4A0913003A43119F49F
:101A0000E7E0E0933003E0E0E0933103E894F2F89C
:101A1000A0913003A33028F0E0913003E150E0932F
:101A20003003AB2D0E94BE25AA2DEAE00E94E32BD5
:101A3000E02131F0E0E0E0933103E4E1E0933003B2
:101A4000EAE0EA1510F4E894F3F80E9405240E94F5
:101A50000B240E94C52BE02109F48DC26894F3F891
:101A6000AE81A13049F4A0911203A13028F4E09195
:101A70001203EF5FE0931203AE81A23049F4A0910C
:101A80001303A23328F4E0911303EB5FE0931303F5
:101A9000AE81A33049F4A0911403A43628F4E09158
:101AA0001403EF5FE0931403AE81A43049F4A091D6
:101AB0001603A83228F4E0911603EF5FE0931603B3
:101AC000AE81A53031F4AC8DA43618F4EC8DEF5F07
:101AD000EC8FAE81A63031F4AD8DA43618F4ED8DC7
:101AE000EF5FED8FAE81A73031F4AE8DA43618F4E0
:101AF000EE8DEF5FEE8FAE81A83049F4A091170311
:101B0000AF3F28F4E0911703EF5FE0931703AE8136
:101B1000AC3049F4A0910F03A03328F4E0910F03F7
:101B2000E45FE0930F03AE81AD3069F4A0913E0312
:101B3000B0913F03A433E8E0BE0728F40E94AC2331
:101B400031960E946C23AE81AE3031F4A88DA4365C
:101B500018F4E88DEB5FE88FAE81AF3031F4A98DDA
:101B6000A43618F4E98DEB5FE98FAE81A03131F432
:101B7000AA8DA43618F4EA8DEB5FEA8FAE81A1310D
:101B800031F4AC89A83C18F4EC89EB5FEC8BAE81A6
:101B9000A23131F4AD89A83C18F4ED89EB5FED8BEF
:101BA000AE81A33131F4AE89A83C18F4EE89EB5F25
:101BB000EE8BAE81A43169F4A0914E03B0914F0336
:101BC000A835E2E0BE0728F40E9422237E960E94F8
:101BD0008A23AE81A53189F4A0910F03EAE0EA9F40
:101BE000F001EA5BFF4FAB85BC85AE17BF0728F459
:101BF000EB85FC853196EB87FC87AE81A63149F4F5
:101C0000A0912903A13028F4E0912903EF5FE0932C
:101C10002903AE81A73149F4A0912B03A23328F404
:101C2000E0912B03EF5FE0932B03AE81A83149F4E1
:101C3000A0912A03A13028F4E0912A03EF5FE093FA
:101C40002A03AE81A93191F4A32FEFE00E94F82579
:101C50000E94C72409F03F5FA32FEEE10E94F82500
:101C6000E1E00E94C52BE02109F03F5FAE81AA317F
:101C700059F40E94FF25AC3BE2E0BE0728F40E9425
:101C8000E82531960E947C23AE81AB3191F40E940D
:101C90005F22A73EE3E0BE07E0E08E07E0E09E079C
:101CA00040F40E942222EF5FFF4F6F4F7F4F0E9450
:101CB0008123AE81AC3161F4A0E023FCA1E0A1302E
:101CC00038F4E0E023FCE1E0EF5F0E944C2D23F8C4
:101CD000AE81AD3169F40E94E221AE3DE3E0BE0782
:101CE00038F40E94C3213A96E0934603F0934703E9
:101CF000AE81AE3169F40E94EC21A835E2E0BE0766
:101D000038F40E94CF213A96E0935203F0935303A4
:101D1000AE81AF3149F4A0910703AA3028F4E091D5
:101D20000703EF5FE0930703AE81A03249F4A0916F
:101D30000903AB3028F4E0910903EF5FE093090356
:101D4000AE81A13249F4A0910A03AB3028F4E091AE
:101D50000A03EF5FE0930A03AE81A23249F4A09137
:101D60000B03AB3028F4E0910B03EF5FE0930B0320
:101D7000AE81A33249F4A0910C03AB3028F4E0917A
:101D80000C03EF5FE0930C03AE81A43249F4A09101
:101D90000D03AB3028F4E0910D03EF5FE0930D03EA
:101DA000AE81A53249F4A0912003A13028F4E0913E
:101DB0002003EF5FE0932003AE81A63249F4A091A7
:101DC0002103A13028F4E0912103EF5FE093210388
:101DD000AE81A73249F4A0912203A13028F4E0910A
:101DE0002203EF5FE0932203AE81A83249F4A09171
:101DF0002303A13028F4E0912303EF5FE093230352
:101E0000AE81A93249F4A0912403A13028F4E091D5
:101E10002403EF5FE0932403AE81AA3249F4A0913A
:101E20002503A33028F4E0912503EF5FE093250319
:101E3000AE81AB3249F4A0912603A13028F4E091A1
:101E40002603EF5FE0932603AE81AC3249F4A09104
:101E50002703A13028F4E0912703EF5FE0932703E5
:101E6000AE81AD3291F40E94F122AF39E6E8BE07AF
:101E7000E1E08E07E0E09E0740F40E94D922E65F91
:101E8000FF4F6F4F7F4F0E94E222AE81AE3259F476
:101E90000E940426A031E7E2BE0728F40E944322F4
:101EA0003A960E944822AE81AF3261F4A0E036FC3F
:101EB000A1E0A13038F4E0E036FCE1E0EF5F0E9401
:101EC0004C2D36F8AE81AC3549F4A0910603AA3FFB
:101ED00028F4E0910603EB5FE0930603AE81AD3595
:101EE00031F4A9A1A73018F4E9A1EF5FE9A3AE810D
:101EF000AE3559F4AF85B889A83BEBE0BE0728F4AE
:101F0000EF85F8893196EF87F88BAE81AF3531F4E4
:101F1000A8A1AA3018F4E8A1EF5FE8A3AE81A0362B
:101F200031F4AF8DAA3018F4EF8DEF5FEF8FAE81F3
:101F3000A13649F4A0911C03AC3328F4E0911C03B2
:101F4000EF5FE0931C03AE81A23649F4A091190320
:101F5000AA3F28F4E0911903E65FE0931903AE81EC
:101F6000A33649F4A0911803AA3F28F4E09118037E
:101F7000E65FE0931803EAE0EB1510F4E894F2F85A
:101F8000AB2DEAE00E94DE2B0E2E0E94D0250E948F
:101F90008D2509F473C26894F2F8AE81A13049F43A
:101FA000A0911203A13028F0E0911203E150E093D8
:101FB0001203AE81A23049F4A0911303AB3028F094
:101FC000E0911303E550E0931303AE81A33049F48D
:101FD000A0911403AD3328F0E0911403E150E09395
:101FE0001403AE81A43049F4A0911603A53128F062
:101FF000E0911603E150E0931603AE81A53031F471
:10200000AC8DA13018F0EC8DE150EC8FAE81A63094
:1020100031F4AD8DA13018F0ED8DE150ED8FAE8132
:10202000A73031F4AE8DA13018F0EE8DE150EE8F77
:10203000AE81A83049F4A0911703A13028F0E091B7
:102040001703E150E0931703AE81AC3049F4A0913F
:102050000F03A93128F0E0910F03EC50E0930F0338
:10206000AE81AD3069F4A0913E03B0913F03AD362F
:10207000E7E0BE0728F00E94AC2331970E946C2352
:10208000AE81AE3031F4A88DA63018F0E88DE55061
:10209000E88FAE81AF3031F4A98DA63018F0E98D0C
:1020A000E550E98FAE81A03131F4AA8DA63018F049
:1020B000EA8DE550EA8FAE81A13131F4AC89A130CF
:1020C00018F0EC89E550EC8BAE81A23131F4AD898A
:1020D000A13018F0ED89E550ED8BAE81A33131F4DC
:1020E000AE89A13018F0EE89E550EE8BAE81A431B7
:1020F00061F4A0914E03B0914F030E94382D28F453
:102100000E9422237E970E948A23AE81A53189F402
:10211000A0910F03EAE0EA9FF001E654F040AB859E
:10212000BC85EA17FB0728F4EB85FC853197EB8724
:10213000FC87AE81A63149F4A0912903A13028F093
:10214000E0912903E150E0932903AE81A73149F4DE
:10215000A0912B03A23028F0E0912B03E150E093F3
:102160002B03AE81A83149F4A0912A03A13028F0B5
:10217000E0912A03E150E0932A03AE81A93119F4DA
:10218000323008F03150AE81AA3159F40E94FF2557
:10219000A935E2E0BE0728F00E94E82531970E94A9
:1021A0007C23AE81AB3191F40E945F22AB30E0E042
:1021B000BE07E0E08E07E0E09E0740F00E9422228A
:1021C000E150F040604070400E948123AE81AC310C
:1021D00059F4A0E023FCA1E0A13030F0A0E023FC02
:1021E000A1E00E94092623F8AE81AD3161F40E947E
:1021F000E2210E94382D38F40E94C3213197E093E8
:102200004603F0934703AE81AE3161F40E94EC21A6
:102210000E94382D38F40E94CF213197E093520369
:10222000F0935303AE81AF3149F4A0910703A2307C
:1022300028F0E0910703E150E0930703AE81A0325C
:1022400049F4A0910903A23028F0E0910903E1507C
:10225000E0930903AE81A13249F4A0910A03A130B1
:1022600028F0E0910A03E150E0930A03AE81A23224
:1022700049F4A0910B03A13028F0E0910B03E15049
:10228000E0930B03AE81A33249F4A0910C03A1307B
:1022900028F0E0910C03E150E0930C03AE81A432EE
:1022A00049F4A0910D03A13028F0E0910D03E15015
:1022B000E0930D03AE81A53249F4A0912003A13033
:1022C00028F0E0912003E150E0932003AE81A63294
:1022D00049F4A0912103A13028F0E0912103E150BD
:1022E000E0932103AE81A73249F4A0912203A130EB
:1022F00028F0E0912203E150E0932203AE81A8325E
:1023000049F4A0912303A13028F0E0912303E15088
:10231000E0932303AE81A93249F4A0912403A130B4
:1023200028F0E0912403E150E0932403AE81AA3227
:1023300049F4A0912503A13028F0E0912503E15054
:10234000E0932503AE81AB3249F4A0912603A1307E
:1023500028F0E0912603E150E0932603AE81AC32F1
:1023600049F4A0912703A13028F0E0912703E15020
:10237000E0932703AE81AD3269F40E94F1220E94FE
:102380003C2D40F40E94D922E150F0406040704062
:102390000E94E222AE81AE3251F40E9404260E94D5
:1023A000382D28F40E94432231970E944822AE81A2
:1023B000AF3259F4A0E036FCA1E0A13030F0A0E04B
:1023C00036FCA1E00E94092636F8AE81AC3549F40E
:1023D000A0910603A13028F0E0910603E550E093B8
:1023E0000603AE81AD3531F4A9A1A13018F0E9A101
:1023F000E150E9A3AE81AE3559F4AF85B889A13D6E
:10240000E7E0BE0728F0EF85F8893197EF87F88B72
:10241000AE81AF3531F4A8A1A13018F0E8A1E150A8
:10242000E8A3AE81A03631F4AF8DA13018F0EF8D66
:10243000E150EF8FAE81A13649F4A0911C03A13089
:1024400028F0E0911C03E150E0931C03AE81A2361A
:1024500049F4A0911903AB3028F0E0911903EA5038
:10246000E0931903AE81A33649F4A0911803A1307B
:1024700028F0E0911803EA50E093180323FC24C0ED
:10248000E0912E03A6ECB3E0FF27662777270E9492
:102490003C2A0E94DC2C0E9410260E943C2D3CF419
:1024A0000E9419260E9422260E94292609C0E0E0E7
:1024B000E093B603E093B703E093B803E093B90366
:1024C0000E9432260E94362623FE4CC0EF81F885FA
:1024D0000E944B250E94E62C0E94E12CE0E0F0E0F7
:1024E00060E874E40E94142BA0E0B0E48CE995E469
:1024F0000E94C62ADF01CB01EF85F889662777277E
:102500000E943C2A0E943E22DF01CB01E3E3F3E379
:1025100065E872E40E94142BE093C603F093C703AE
:102520006093C8037093C903A0911003A13048F4CD
:10253000E0E0E093C603E093C703E093C803E093B1
:10254000C9030E9419260E942926E0910703A09141
:102550000803AE1738F00E9432260E943626E0E0CB
:10256000E0930803F0915403E0E0DF01E0912F03D2
:10257000F0E0EA0FFB1FA6E9B3E00E94C8210E9429
:102580003A26A0E0B0E080E192E40E94142B7F9311
:102590006F93FF93EF930E94FF250E944326AF9114
:1025A000BF918F919F91662777270E943C2A0E94B6
:1025B000C62AE0939603F093970360939803709371
:1025C00099030E944826E0E0F0E060E87FE30E9483
:1025D0007F2B0E2E0E944826E0E0F0E068EC72E4CB
:1025E0000E94792BE021E9F00E943A260E942226DF
:1025F000AEE7B3E00E94052A0E94DC2C0E943A2636
:10260000E0939A03F0939B0360939C0370939D0364
:102610000E9448260E947823A0E4B3E00E94FA2199
:1026200015C0E0E0E0937E03E0937F03E093800336
:10263000E0938103E0939A03E0939B03E0939C0370
:10264000E0939D03E0934003E09341030E948322C3
:102650000E94FA220E947F2BEF930E9451260E9433
:102660007F2BAF91EA23C1F10E941022E0E0F0E05D
:1026700068EC72E40E94142B0E945F220E94EB2CF3
:102680000E943E220E945326A0919203B091930390
:102690008091940390919503E0E0F0E064E172E4AE
:1026A0000E94C62ADF01CB010E949A220E94142BAD
:1026B000A0E0B0E080E291E40E94C62A0E94532686
:1026C000E0919203F09193036091940370919503CC
:1026D000DE0114960E9477220E94A324A0911A037F
:1026E000EDEF0E94DE2B0E220E94A924E02129F0AA
:1026F000E0911A03EF5FE0931A03A62D0E94BE2516
:10270000A0911A03EFEF0E94DE2B0E220E94A92453
:10271000E02129F0E894F0F8E0E0E0931A03A091BA
:102720001A03EEE10E94C52B0E2E0E94A924E0217F
:1027300019F0E1E0E0931D03E0911C03E03019F48F
:10274000E0E0E0931D030E9408230E94FA220E9409
:10275000102C0E949425A0911D03E0E00E94E32B21
:10276000E02119F0E1E0E0931D03A0911D03AC33DB
:1027700009F41FEFA0910603A13028F0E0910603B1
:10278000F0E00E94C8234420C9F4E02FF0E0349622
:102790000E94CD23AE0FBF1FE12F0E945C26A4E054
:1027A0000E94A421A02F0E946626A09134030E94BB
:1027B000A421A12F0E94A4210E946B26E1E0E41530
:1027C00009F057C04424A09114030E947426E0939A
:1027D0001503F0E0BC96DF01E0911103F0E0AE0FCD
:1027E000BF1FE0911203F0E0AE0FBF1FE091130393
:1027F000F0E0AE0FBF1FE0911603F0E0AE0FBF1F79
:10280000EC8DF0E0AE0FBF1FED8DF0E0AE0FBF1FFF
:10281000EE8DF0E0AE0FBF1FE09117030E945C2623
:10282000ACE20E94A421A09111030E94A421A091D6
:1028300012030E94A421A09113030E94A421A0913D
:1028400015030E94A421A09116030E94A421AC8D1F
:102850000E94A421AD8D0E94A421AE8D0E94A421CE
:10286000A09117030E946626A0E00E9466260E949F
:102870006B26233608F06AC50E94E2252081A0E07D
:10288000F799A1E0EA2FE295E07F0E2EA0E0F39900
:10289000A1E0EA2FEE0FEE0F0E0EA0E0F499A1E0FA
:1028A000EA2FEE0FA02DAE0FE0E0F599E1E0EA0F80
:1028B000EAA3EAE0EFABE8AFE9AFEAAFEBAFECAF2A
:1028C000EDAF0E947A26EAE00E948226EAE00E94AA
:1028D0008726EAE00E948C26EAE00E949126EAE040
:1028E000DE01AB5BBF4FEC93E89435F8E091250334
:1028F000E03021F40E949626E00DEBA3A091250381
:10290000A13081F4A0E022FCA1E0EA2FEE0FE75F06
:102910000E2EA0E022FCA1E0EA2FEE0FEE0FE00D5C
:102920000E94AF26A0912503A23099F40E9496261A
:102930000E0EA0E022FCA1E0EA2F0E94C9260E0E96
:10294000A0E022FCA1E0EA2FE295E07FEE0FE00D8F
:10295000EBA3A0912503A33031F4E0E022FCE1E0F9
:10296000E85F0E94AF26A0910F03A83109F041C093
:102970000E94CE26A23DE0E0BE07E0E08E07E0E048
:102980009E071CF0E1E0E09301030E94DC26A83FD3
:10299000E0E0BE07E0E08E07E0E09E071CF0E3E029
:1029A000E09301030E94DC26AF3FE0E0BE07E0E0D9
:1029B0008E07E0E09E071CF0E7E0E09301030E9431
:1029C000DC26A430E1E0BE07E0E08E07E0E09E07F1
:1029D0001CF0EFE0E09301030E94DC26AE30E1E062
:1029E000BE07E0E08E07E0E09E071CF0EFE1E09319
:1029F0000103A0910F03A43209F041C00E94CE262A
:102A0000A633E1E0BE07E0E08E07E0E09E071CF0A1
:102A1000E1E0E09301030E94DC26AA34E1E0BE0776
:102A2000E0E08E07E0E09E071CF0E3E0E0930103A6
:102A30000E94DC26AE35E1E0BE07E0E08E07E0E074
:102A40009E071CF0E7E0E09301030E94DC26A83615
:102A5000E1E0BE07E0E08E07E0E09E071CF0EFE05B
:102A6000E09301030E94DC26AC37E1E0BE07E0E022
:102A70008E07E0E09E071CF0EFE1E0930103A091D8
:102A80000F03A03309F041C00E94CE26A638E1E032
:102A9000BE07E0E08E07E0E09E071CF0E1E0E09377
:102AA00001030E94DC26AC3CE1E0BE07E0E08E07BB
:102AB000E0E09E071CF0E3E0E09301030E94DC26C7
:102AC000A63DE1E0BE07E0E08E07E0E09E071CF0D7
:102AD000E7E0E09301030E94DC26A03EE1E0BE07B0
:102AE000E0E08E07E0E09E071CF0EFE0E0930103DA
:102AF0000E94DC26AF3EE1E0BE07E0E08E07E0E0AA
:102B00009E071CF0EFE1E09301030E9408230E945E
:102B1000E5262CF00E94ED260E94F326E9AF0E94E4
:102B2000ED260E94A72CEAAFA0917103AA2382F49C
:102B3000A0917003B0917103A73FEFEFBE071CF4A3
:102B4000689435F802C0E0E4EFAB0E94FE2602C0B4
:102B5000E89435F80E9409271A972CF00E940E2756
:102B60000E941227EFAB0E940E270E94952CE8AF1F
:102B70000E94DC260E941A270E94F326EBAF0E94D7
:102B80001F270E94F326ECAF0E941F270E94A72C4C
:102B9000EDAF0E94DC260E9425273CF4E0E4EBAF79
:102BA000ECAFEDAFE0E0E0930103213009F04CC061
:102BB0000E942D270E943727A83EE3E0BE0788F039
:102BC000ECA1E05EECA30E943C270E9441270E94FA
:102BD0004D270E9452270E945E270E944326DF0154
:102BE00015C0ECA1E056ECA30E943727A436E0E024
:102BF000BE0720F00E943C270E9452270E944D27CA
:102C00000E9443260E9463270E945E27EAE0F0E0CC
:102C10000E946B27A0910003AA3010F0E2E0EEAF13
:102C2000A09100030E947027EFAF0E947627AC2D81
:102C3000B0E00E947B270E947E273B96BF01AC2D0F
:102C40000E947027DB01EC93223009F075C0ECA1E3
:102C5000E05CECA30E94F122A03AE6E8BE07E1E0C6
:102C60008E07E0E09E0780F0FE01F6963A96FF930D
:102C7000EF930E94F122E0EAF6E861E070E00E9442
:102C80008327AF91BF91EC930E94F1220E948E277F
:102C900080F0FE01F6963B96FF93EF930E94F1229F
:102CA000E0E1F7E260E070E00E948327AF91BF911E
:102CB000EC930E94F1220E94962770F0FE01F69696
:102CC0003C96FF93EF930E94F1220E949E240E9463
:102CD0008327AF91BF91EC930E94F1220E94252798
:102CE00070F0FE01F6963D96FF93EF930E94F1225D
:102CF0000E941A270E948327AF91BF91EC930E94F4
:102D0000F1220E94E52660F0FE01F6963E96FF93C2
:102D1000EF930E949E270E948327AF91BF91EC936F
:102D2000FE01F6963F96FF93EF930E949E270E9426
:102D3000A32CAF91BF91EC93233009F096C0E7E745
:102D40000E94A427A0918D03AA2392F4E0918A0304
:102D5000F0918B0360918C0370918D030E94932BF3
:102D6000E0938A03F0938B0360938C0370938D033D
:102D70000E9451260E943E2277231AF4E0E40E942A
:102D800091260E9451260E943E220E94AB2718F4F1
:102D9000E0E40E948C260E9451260E943E220E945E
:102DA000B42718F4E0E40E9487260E9451260E946E
:102DB0003E220E94BD2718F4E0E40E9482260E9471
:102DC000C0270E948E2784F0FE01F6963B96FF9363
:102DD000EF930E94C027E0E1F7E260E070E00E941C
:102DE000F326AF91BF91EC930E94C0270E949627D3
:102DF00074F0FE01F6963C96FF93EF930E94C02775
:102E00000E949E240E94F326AF91BF91EC930E94F2
:102E1000C0270E94252764F0FE01F6963D96FF9399
:102E2000EF930E94C0270E94C927AF91BF91EC93F6
:102E30000E94C0270E94E52664F0FE01F6963E96A9
:102E4000FF93EF930E94CB270E94F326AF91BF918F
:102E5000EC93FE01F6963F96FF93EF930E94CB27EB
:102E60000E94A72CAF91BF91EC93243009F059C078
:102E70000E94D127A0916D03AA2312F40E94D627A5
:102E80000E94E12777231AF4E0E40E9491260E9431
:102E9000E1270E94AB2718F4E0E40E948C260E94F0
:102EA000E1270E94B42718F4E0E40E9487260E94DC
:102EB000E1270E94BD2718F4E0E40E9482260E94C8
:102EC000E727A031E7E2BE0734F00E94EC270E941A
:102ED000F127DB01EC930E94E727A83EE3E0BE0761
:102EE00034F00E94F5270E94FA27DB01EC930E9440
:102EF000E727A436E0E0BE0734F00E94FE270E94D8
:102F00000328DB01EC930E94E7271A9744F00E9404
:102F100007280E94E7270E947B27DB01EC930E9491
:102F20000C28253071F50E94D127E0E50E94822609
:102F3000A091BD03AA231AF4E0E40E948C260E940B
:102F40008322E0E0F0E060E171E40E94592B18F484
:102F5000E0E40E9487260E941828A436E0E0BE071D
:102F600034F00E94FE270E941D28DB01EC930E9492
:102F700007280E9418280E947B270E947E270E9413
:102F800021282630D9F5ECA1E058ECA3E0E0EFAF22
:102F9000E5E00E942B28E8E70E948226AC81BD81F3
:102FA000A83EE3E0BE0754F00E94F527AC81BD8146
:102FB000E8EEF3E00E941227DB01EC93AC81BD81C7
:102FC000A436E0E0BE0754F00E94FE27AC81BD812C
:102FD000E4E6F0E00E941227DB01EC930E94072850
:102FE000AC81BD810E947B270E947E273F96BF0156
:102FF000AC81BD810E943028DB01EC93273009F0C1
:1030000051C0113058F1ECE0EFAFA12F0E947426AF
:10301000E436A0E0FA0754F00E947627A12FB0E032
:10302000E8ECF0E00E941227DB01EC93A12F0E9454
:1030300074263A9754F00E94EC27A12FB0E0E4E107
:10304000F0E00E941227DB01EC930E94F527A12FEC
:103050000E947426DF010E94302822C0EBE0EFAF0F
:103060000E943528E436A0E0FA0740F00E94762757
:10307000A985BA85E8ECF0E00E943A280E9435283C
:103080003A9740F00E94EC27A985BA85E4E1F0E088
:103090000E943A280E94F5270E9435280E943D2868
:1030A000DB01EC93283009F079C00E942D27A09114
:1030B0006803B0916903A135EBEFBE0734F4E1E595
:1030C000FBEFE0936803F0936903A0916803B0916C
:1030D0006903A03BE4E0BE0734F0EFEAF4E0E093DC
:1030E0006803F0936903A0916903AA2352F4E0E412
:1030F0000E948726E0916803F09169030E948F2B5C
:1031000004C0E0916803F0916903E0936A03F093CF
:103110006B03A0916A03B0916B03ECE3F0E00E94B3
:10312000632CE0934803F09349030E944328ECE3A7
:103130000E94402CA0916A03B0916B03AE1BBF0BA1
:10314000A0934A03B0934B0324FE1DC00E94432862
:103150001A9710F0E2E0EEAF0E9443280E94482840
:10316000EFAF0E947627A0914A03B0914B030E94D3
:1031700043260E9463270E94EC27A0914A03B09146
:103180004B030E944D28E3E70E948C26E8E30E944F
:103190009126E4E5DE01AB5BBF4FEC93293009F0EB
:1031A00059C00E945028A0916D03AA2312F40E94D6
:1031B000D6270E94E12777231AF4E0E40E949126A3
:1031C0000E94E1270E94AB2718F4E0E40E948C26BD
:1031D0000E94E1270E94B42718F4E0E40E948726A9
:1031E0000E94E1270E94BD2718F4E0E40E94822695
:1031F0000E94E727A031E7E2BE0734F00E94EC27E7
:103200000E94F127DB01EC930E94E727A83EE3E050
:10321000BE0734F00E94F5270E94FA27DB01EC93E9
:103220000E94E727A436E0E0BE0734F00E94FE27A4
:103230000E940328DB01EC930E94E7271A9744F0D1
:103240000E9407280E94E7270E947B27DB01EC935E
:103250000E940C282A30D9F40E945028E0E50E94F0
:1032600082260E941828A436E0E0BE0734F00E94AF
:10327000FE270E941D28DB01EC930E9407280E9474
:1032800018280E947B270E947E270E9421282B302D
:1032900069F5ECA1E054ECA30E9457280E94042693
:1032A000A83EE3E0BE0730F00E94F5270E94042606
:1032B0000E9441270E940426A436E0E0BE0730F0B9
:1032C0000E94FE270E9404260E9452270E9407287F
:1032D0000E9404260E9443260E946327FE01F69660
:1032E0003F96BF010E9404260E944D28AA89A13062
:1032F00030F1ECA1EF77ECA3E0912D03E170EE0F3C
:10330000ABA1EA23EBA3E058EBA30E947A26E9E7FE
:103310000E948226E0E50E948726E0E50E948C2636
:103320000E940728AA89B0E00E947B270E947E277E
:103330003F96BF01AA890E947027DB01EC93F29BA4
:1033400005C0EBA1EB7FEBA3EF5FEBA3233609F006
:10335000C2C451E0503140F40E945B28EAE0EC9393
:10336000E89435F85F5FF6CFAE81EBE50E94622806
:10337000EAE50E94C52BE02911F0EFE2EE83AE8171
:10338000A03311F4ECE5EE83EE81E03029F4E09116
:103390001103F0E0ED87FE87AE81A13029F4E091C2
:1033A0001203F0E0ED87FE87AE81A23029F4E091B0
:1033B0001303F0E0ED87FE87AE81A33029F4E0919E
:1033C0001403F0E0ED87FE87AE81A43029F4E0918C
:1033D0001603F0E0ED87FE87AE81A53021F4EC8D79
:1033E000F0E0ED87FE87AE81A63021F4ED8DF0E0B0
:1033F000ED87FE87AE81A73021F4EE8DF0E0ED87FA
:10340000FE87AE81A83029F4E0911703F0E0ED8744
:10341000FE87AE81A93019F4E0E0ED87EE87AE813A
:10342000AA3019F4E0E0ED87EE87AE81AB3019F4F5
:10343000E0E0ED87EE87AE81AC3029F4E0910F0338
:10344000F0E0ED87FE87AE81AD3021F40E94AC2321
:10345000ED87FE87AE81AE3021F4E88DF0E0ED8798
:10346000FE87AE81AF3021F4E98DF0E0ED87FE8775
:10347000AE81A03121F4EA8DF0E0ED87FE87AE81C8
:10348000A13121F4EC89F0E0ED87FE87AE81A23115
:1034900021F4ED89F0E0ED87FE87AE81A33121F4C0
:1034A000EE89F0E0ED87FE87AE81A43121F40E9421
:1034B0002223ED87FE87AE81A53121F4EB85FC85C3
:1034C000ED87FE87AE81A63129F4E0912903F0E073
:1034D000ED87FE87AE81A73129F4E0912B03F0E060
:1034E000ED87FE87AE81A83129F4E0912A03F0E050
:1034F000ED87FE87AE81A93121F4E32FF0E0ED875F
:10350000FE87AE81AA3121F40E94E825ED87FE876F
:10351000AE81AB3131F4E0915E03F0915F03ED8752
:10352000FE87AE81AC3131F4E0E023FCE1E0F0E075
:10353000ED87FE87AE81AD3121F40E94C321ED8776
:10354000FE87AE81AE3121F40E94CF21ED87FE8748
:10355000AE81AF3129F4E0910703F0E0ED87FE87FB
:10356000AE81A03229F4E0910903F0E0ED87FE87F7
:10357000AE81A13229F4E0910A03F0E0ED87FE87E5
:10358000AE81A23229F4E0910B03F0E0ED87FE87D3
:10359000AE81A33229F4E0910C03F0E0ED87FE87C1
:1035A000AE81A43229F4E0910D03F0E0ED87FE87AF
:1035B000AE81A53229F4E0912003F0E0ED87FE878B
:1035C000AE81A63229F4E0912103F0E0ED87FE8779
:1035D000AE81A73229F4E0912203F0E0ED87FE8767
:1035E000AE81A83229F4E0912303F0E0ED87FE8755
:1035F000AE81A93229F4E0912403F0E0ED87FE8743
:10360000AE81AA3229F4E0912503F0E0ED87FE8730
:10361000AE81AB3229F4E0912603F0E0ED87FE871E
:10362000AE81AC3229F4E0912703F0E0ED87FE870C
:10363000AE81AD3231F4E0915A03F0915B03ED8736
:10364000FE87AE81AE3221F40E944322ED87FE87D1
:10365000AE81AF3231F4E0E036FCE1E0F0E0ED873E
:10366000FE87AE81AC3529F4E0910603F0E0ED87EA
:10367000FE87AE81AD3521F4E9A1F0E0ED87FE874C
:10368000AE81AE3521F4EF85F889ED87FE87AE81F6
:10369000AF3521F4E8A1F0E0ED87FE87AE81A036DA
:1036A00021F4EF8DF0E0ED87FE87AE81A13629F49D
:1036B000E0911C03F0E0ED87FE87AE81A23629F48D
:1036C000E0911903F0E0ED87FE87AE81A33629F47F
:1036D000E0911803F0E0ED87FE87AE81E0E00E9404
:1036E0006228E3E00E946728E1E10E946728E2E1A6
:1036F0000E946728E3E10E946728E5E10E946728AD
:10370000EBE10E946728EDE10E946728EEE20E944B
:10371000C52BE02911F0F69A01C0F698A0E0F699C1
:10372000A1E0EA2FE795E0E0E795ECA3E0E0EBA36A
:10373000EAA3E0930103AE81B0E0A7FDBFEF0E94D2
:103740007B27E9AFAE81B0E0A7FDBFEF0E94302834
:10375000EAAFAD85BE85A031E7E2BE0740F00E942A
:10376000EC27AD85BE85E0E1F7E20E943A28AD8501
:10377000BE85A83EE3E0BE0730F00E94F527AD8588
:10378000BE850E944127AD85BE85A436E0E0BE0718
:1037900030F00E94FE27AD85BE850E945227AD8580
:1037A000BE851A9730F00E9407280E946C280E945C
:1037B0006327FE01F6963F96BF01AD85BE850E9448
:1037C0004D28EE81E03079F4EDE6EBAFE9E7ECAFC0
:1037D000E8E7EDAFEDE60E942B28E4E50E948226A3
:1037E000E0E50E948726AE81E1E10E946228E2E1E5
:1037F0000E946728E3E10E946728E5E10E946728AC
:10380000EDE10E946728EEE20E94C52BE02931F02D
:103810000E9407280E946C280E946327E7EAE09331
:103820007A00A7E00E949E230E94C823E7E2E0936B
:103830007A000E946F28EEE00E946728E1E10E9472
:10384000C52BE02911F0E1E07E2EAE810E9400241C
:10385000AE81EFE00E946728E2E10E94C52BE029DB
:1038600011F0E2E07E2EAE81E7E00E946228E0E106
:103870000E9467280E94722811F0E3E07E2E0E94C9
:10388000CD23D39708F457C00E9415240E941A2410
:10389000E72D0E94212420F0E8ECF0E00E94C823EC
:1038A000E72D0E9431240E947728AC91A13008F4C2
:1038B00041C00E947E280E9451240E94472D4CF452
:1038C0000E9477280E9487280E94852B0E949228B8
:1038D00023C00E949B280E947324EF930E949B2880
:1038E0000E947C24AF91EA2379F00E9477280E94FD
:1038F00087280E948A2BA0937A03B0937B0380933E
:103900007C0390937D0308C00E949B280E9485241D
:103910001CF00E949D280EC0A0917A03B0917B03F9
:1039200080917C0390917D030E949E240E948D2CA7
:103930000E94C82304C00E94FA230E949D28AE81E1
:10394000AD3051F40E94A5280E94C9270E94AE28DC
:103950000E94B528E0E2EAA3AE81A53151F40E94AD
:10396000A5280E94C9270E94AE280E94B528E0E63B
:10397000EAA30E946F28EEE00E946728E1E10E941E
:10398000C52BE029A9F00E94BF28E4E00E94C328CB
:1039900018F00E94C928EBAF0E94CD231A9728F097
:1039A0000E94CF280E943D28ECAF0E94D128EDAFA5
:1039B000AE810E940024AE81EFE00E946728E2E120
:1039C0000E94C52BE029A9F00E94BF28E2E00E94D6
:1039D000C32818F00E94C928EBAF0E94CD231A9784
:1039E00028F00E94CF280E943D28ECAF0E94D128E9
:1039F000EDAFAE81E7E00E946228E0E10E94672817
:103A00000E947228A9F00E94BF28E1E00E94C3280A
:103A100018F00E94C928EBAF0E94CD231A9728F016
:103A20000E94CF280E943D28ECAF0E94D128EDAF24
:103A3000AE81A43189F40E94D3280E94D828EBAF2C
:103A40000E94D3280E9443260E943D28ECAF0E948A
:103A5000D3280E944828EDAFAE81A63129F40E94F8
:103A6000DD28EBE00E948726AE81A73129F40E9471
:103A7000DD28E0E40E948726AE81A83129F40E9467
:103A8000DD28ECE00E948726AE81A93191F4A09157
:103A9000C903AA2312F40E94FE260E940E270E9448
:103AA0001227EBAF0E940E270E94952CECAFE7E7A0
:103AB000EDAFAE81AA3189F40E94E3280E94D82894
:103AC000EBAF0E94E3280E9443260E943D28ECAF02
:103AD0000E94E3280E944828EDAFAE81AB3171F41B
:103AE000ECE7EFAFE7E70E942B28E8E70E94822689
:103AF0000E9407280E946C280E946327AE81EDE196
:103B00000E946228EEE10E94C52BE029F9F0E3E76C
:103B1000EFAFE8E30E942B28AE81AD3111F4EEE562
:103B200001C0E8E7DE01AF5BBF4FEC930E94E828DD
:103B30001A9738F00E94E8280E9443260E943D28E8
:103B4000ECAF0E94E8280E944828EDAF0E946F2841
:103B5000E6E00E946728E7E00E94C52BE02911F00B
:103B6000E3E7EFAFAE81EEE00E946228EFE00E9453
:103B70006728E0E10E94C52BE02941F0EDE6EFAFB8
:103B8000E9E70E942B28E4E50E948226AE81E1E16C
:103B90000E946228E2E10E9467280E94722819F0C0
:103BA000E8E70E942B28AE81EFE10E94D92B0E2E70
:103BB000E5E20E94D42BE02139F0EDE6EBAFE8E539
:103BC000ECAFEE81EF51EDAFAE81AD3219F4ECA167
:103BD000E05CECA3AE81AE3211F40E945728AE81B6
:103BE000AD35A9F5E7E70E948726EEE50E948C2611
:103BF000E9E30E949126FE01F6963F96A9A1A083D3
:103C0000E7EAE0937A000E949723E0933603F0936B
:103C10003703E7E2E0937A000E94ED28A436E0E063
:103C2000BE0728F00E94ED280E94D828EBAF0E9422
:103C3000ED281A9738F00E94ED280E9443260E9432
:103C40003D28ECAF0E94ED280E944828EDAFAE81E0
:103C5000AE3561F50E9410260E94FF22A2E7B3E074
:103C60000E947722A091C903AA2352F4E091720323
:103C7000F09173030E948F2BE0937203F093730310
:103C80000E940927E4E6F0E00E941227EBAF0E94B1
:103C90000E270E941227ECAF0E940E270E94952C3F
:103CA000EDAFEEE5EFAFE1E00E942B28AE81AF353E
:103CB00029F4EEE5EFAFE2E00E942B28AE81A036BA
:103CC00029F4EEE5EFAFE3E00E942B28AE81A236A7
:103CD00011F4E0E1EAA351E0503108F077C00E940E
:103CE0005B28EC91E03021F40E945B28EFE3EC9339
:103CF0000E945B28AC91A63021F40E945B28EDE77E
:103D0000EC930E945B28AC91A13021F40E945B28C7
:103D1000E6E0EC930E945B28AC91A23021F40E9473
:103D20005B28EBE5EC930E945B28AC91A33021F477
:103D30000E945B28EFE4EC930E945B28AC91A430D6
:103D400021F40E945B28E6E6EC930E945B28AC918C
:103D5000A53021F40E945B28EDE6EC930E945B28DD
:103D6000AC91A73021F40E945B28E7E0EC930E941D
:103D70005B28AC91A83021F40E945B28EFE7EC931C
:103D80000E945B28AC91A93021F40E945B28EFE6E9
:103D9000EC930E945B28AC91AA3021F40E945B282E
:103DA000E0E0EC930E945B28AC91AB3021F40E94E0
:103DB0005B28E1E0EC930E945B28AC91AC3021F4ED
:103DC0000E945B28E8E0EC935F5F86CFE0910103FF
:103DD000E695E6950E94F228EBAD0E94F828EBAD3F
:103DE0000E940029EBAD0E940B29EBAD0E94122925
:103DF000EBAD0E941929EBAD0E942029EBAD0E948A
:103E00002729EEA3E0910103E695E695E6950E9449
:103E1000F228ECAD0E94F828ECAD0E940029ECAD30
:103E20000E940B29EDAD0E941229EDAD0E941929C7
:103E3000EDAD0E942029EDAD0E942729EFA3E0916E
:103E40000103E6950E94F228EDAD0E94F828EDAD41
:103E50000E940029EDAD0E940B29ECAD0E941229B1
:103E6000ECAD0E941929ECAD0E942029ECAD0E9416
:103E70002729E8A7EEAD0E94F228EFAD0E94F828AE
:103E8000EFAD0E940029EFAD0E940B29ECA10E942A
:103E90001229ECA10E941929ECA10E942029E0918D
:103EA0000103E170EA2BE9A70E942D290E94F22864
:103EB0000E942D290E9432290E942D290E94382912
:103EC0000E942D290E9441290E944B290E942D29E0
:103ED0000E944F290E942D290E9458290E942D29B5
:103EE000E295E170EA2BEAA70E9461290E94F2287C
:103EF0000E9461290E9432290E9461290E9438296A
:103F00000E9461290E944129E2950E9412290E9483
:103F100066290E944F290E9466290E9458290E9402
:103F20006629E295E170EA2BEBA7ECA10E946B29D0
:103F30000E9461290E94F8280E9461290E9400299C
:103F40000E9461290E940B290E946F290E94122958
:103F50000E946F290E9419290E946F290E9420291E
:103F60000E946F290E942729ECA70E9466290E94BF
:103F7000F2280E9466290E9432290E9466290E9426
:103F800038290E9466290E9441290E9474290E94B2
:103F900012290E946F290E944F290E946F290E94B6
:103FA00058290E946F29E295E170EA2BEDA70E9443
:103FB00079290E94F2280E9479290E9432290E94C0
:103FC00079290E9438290E9479290E944129EE1FEF
:103FD000E0E0EE1F0E9412290E947E290E944F29D4
:103FE0000E947E290E9458290E947E29E295E17054
:103FF000EA2BEEA7EBA1E2950E94F2280E94792914
:104000000E94F8280E9479290E9400290E9479299B
:104010000E940B29EFAD0E941229EFAD0E941929D1
:10402000EFAD0E942029EFAD0E942729EFA70E9443
:104030007E290E94F2280E947E290E9432290E9435
:104040007E290E9438290E947E29E695E695E6950C
:104050000E9483290E2EA0E035FCA1E0EA2FEE0F8E
:10406000EE0FEE0FE029AE2FEFA9E2950E9488290E
:10407000EFA90E945829EFA9E295EF70E695E1704B
:10408000EA2BE8ABEFA9E695E695E6950E94F228C3
:10409000EFA9E695E6950E948E29EFA90E94932943
:1040A000EFA90E948329AE2FEBA10E944B29EBA11F
:1040B0000E949B29EBA10E949E29EBA1E695E1704D
:1040C000EA2BE9ABEBA10E946B29E8ADE2950E94D7
:1040D0008E29E8AD0E940029E8AD0E94A329AE2FE9
:1040E000E8AD0E944B29E8AD0E949B29E8ADE6951A
:1040F0000E949E29E8ADE170EA2BEAABEBA10E9499
:1041000074290E94F228EAA10E948E29EAA10E9445
:104110009329EAA1E695E6950E948329AE2FE091C6
:104120000103E2950E941229EBA1EE1FE0E0EE1FD1
:104130000E948829EAA1E695E695E6950E949E29C7
:10414000EAA1E295E170EA2BEBABEAA10E946B29B0
:10415000E9ADE2950E948E29E9AD0E940029E9AD02
:104160000E94A329AE2FEAAD0E944B29EAAD0E941E
:104170009B29EAADE6950E949E29EAADE170EA2B03
:10418000ECABEAA10E9474290E94F228EAADE29504
:104190000E948E29EAAD0E940029EAAD0E94A3295F
:1041A000AE2FE9AD0E944B29E9AD0E949B29E9ADF4
:1041B000E6950E949E29E9ADE170EA2BEDAB33FE56
:1041C0000DC051E0513150F4E52FF0E0DE0195963D
:1041D000AE0FBF1FEFEFEC935F5FF4CF0E94A729F4
:1041E0005D3078F40E94AD29A2E5B8E00E94A32BCF
:1041F000E17011F45D9801C05D9A0E94B4295F5F7F
:10420000EFCF0E94BC295D3078F40E94AD29A0E375
:10421000B8E00E94A32BE17011F45D9801C05D9A93
:104220000E94B4295F5FEFCF0E94BC295D3078F413
:104230000E94AD29A2E0B8E00E94A32BE17011F426
:104240005D9801C05D9A0E94B4295F5FEFCF0E9424
:10425000BC295D3078F40E94AD29A6E0B8E00E9448
:10426000A32BE17011F45D9801C05D9A0E94B429FE
:104270005F5FEFCF0E94BC295A3098F45E9885E2C8
:104280008A95F1F7E9E0E51BA0E4B1E00E94A32BD9
:10429000E17011F45D9801C05D9A0E94B4295F5FDE
:1042A000EBCF41E04131E8F451E05930C0F45E9881
:1042B00085E28A95F1F7E42FF0E0DE019596AE0FE6
:1042C000BF1FAC91E8E0E51B0E949B2BE17011F44D
:1042D0005D9801C05D9A0E94B4295F5FE6CF4F5F91
:1042E000E1CF5D9A85E28A95F1F7289A8DEC9AE004
:1042F0000197F1F70E94A324A92DEAE00E94DE2B8A
:104300000E2AAB2DEAE00E94DE2B0E2AAA2DEAE04F
:104310000E94DE2BE02929F0E0E0E0935003E093D7
:104320005103A82DE4E60E94E32B0E2EA0E0F099A5
:10433000A1E00E94C72429F00E942723F09AE89464
:1043400033F80C94AD05FFCFAA93E091C000E07262
:10435000E1F3E881E093C60021960895A0913A0325
:10436000B0913B030895A0919A03B0919B03809173
:104370009C0390919D030895E0E0F0E061EE75E408
:104380000E94142B0895E0914603F091470308958D
:10439000662777270E943C2A0E94DC2C0895E09132
:1043A0005203F09153030895A091A203B091A30387
:1043B0008091A4039091A5030895E0E0F0E060E20D
:1043C00071E40895A0914603B09147030895E0E099
:1043D000F0E00E94FA2B0895A0915203B09153038C
:1043E0000895E091CA03F091CB036091CC037091E2
:1043F000CD0308950E94032AED93FC930895A091A4
:10440000B603B091B7038091B8039091B903E0E08F
:10441000F0E06AE774E40E94C62ADF01CB01ACCF6A
:10442000A091B203B091B3038091B4039091B5030E
:104430000895A091D603B091D7038091D8039091AD
:10444000D9030895E0915E03F0915F0360916003EA
:10445000709161030895A4E6B0E080E090E00E94CE
:10446000202CDF01CB01E091B203F091B303609106
:10447000B4037091B5030E94EB2C08950E94F02CB8
:104480000E946F2A0895E0915803F091590308950E
:10449000E0935803F09359030895A091D203B0918B
:1044A000D3038091D4039091D5030895E093D20370
:1044B000F093D3036093D4037093D5030895A09130
:1044C0005E03B0915F038091600390916103089552
:1044D0000E94202CDF01CB01E091D203F091D303A5
:1044E0006091D4037091D5030E94EB2CC7CF0E943A
:1044F000052AED93FC930895E0E0F0E061EE75E4A9
:104500000E94C62A0895A091BA03B091BB0380917E
:10451000BC039091BD030895E0E0F0EC69E774EC12
:104520000E94592B0895E7EEF3E0E0937403F093B3
:1045300075030895E091BA03F091BB036091BC0349
:104540007091BD030895E091BE03F091BF036091A7
:10455000C0037091C1030895A0919E03B0919F0381
:104560008091A0039091A1030895E0939E03F0939E
:104570009F036093A0037093A1030895A091A603E5
:10458000B091A7038091A8039091A9030895E091A9
:104590009E03F0919F036091A0037091A103089581
:1045A000A091AE03B091AF038091B0039091B1039D
:1045B0000895E0915A03F0915B0360915C03709160
:1045C0005D030895E0935A03F0935B0360935C03EB
:1045D00070935D030895EDDFAEE3B0E00E94112D0E
:1045E0000895A0915A03B0915B0380915C03909170
:1045F0005D030895E0E0F0E060E070E00895DDDE46
:104600000E94C62A0895E0E00E94E32B0E2E089532
:10461000A0917E03B0917F038091800390918103EC
:1046200008950E22A0911D03ECE30E94DE2B089555
:10463000A0915003B09151030895A0914E03B09101
:104640004F03C5CEE0914E03F0914F030895A4E6C9
:10465000B0E00C94C629E7EAE0937A00A4E00E9457
:104660008603EF2FF0E06E2EE7E2E0937A000895E4
:10467000E7EAE0937A00A3E00E948603EF2FF0E0E0
:104680009E2EE7E2E0937A000895E7EAE0937A004D
:10469000A1E00E948603EF2FF0E0BE2EE7E2E09358
:1046A0007A000895E0E0F0E00E94192D0895EBE013
:1046B000E093DF03E8EBE093E0030895E8ECF0E03B
:1046C000E0936403F09365030895E0EDF7E0E09371
:1046D0006603F09367030895E0933E03F0933F036E
:1046E00008950E94BB2B0E943C2A0E94DC2C089556
:1046F00064DE0E94142B0895E0934403F093450375
:104700000895E0935E03F0935F03609360037093FA
:1047100061030895E0934E03F0934F030895AAE0D8
:10472000B0E00E94C629E7EAE0937A0008950E946B
:1047300086030E94B02B0E94AC2B08950E94860332
:10474000EF2FF0E00895E0938203F09383036093EA
:104750008403709385030895E0913E03F0913F0335
:104760000895E0918203F091830360918403709136
:1047700085030895E7E2E0937A008AE48A95F1F7E9
:1047800008958AE48A95F1F7E7EAE0937A000895BC
:10479000E0933403F09335030895A0913403B0916E
:1047A00035030895FADFEAEFF0E00895F6DFEEE171
:1047B000F0E00E94F42B08950E2EA52DE1E00E945A
:1047C000E32B0E22AA89E5E00E94DE2BE02108956A
:1047D000AA89E5E00E94C52B0E2EAE81ECE5089576
:1047E000E0211E2EAA89E7E00E94C52B0E2EAE8185
:1047F000ECE50895E0E0E0933403E0933503089599
:10480000E6E00E94C52B0E2E0895AA2DEAE00E9434
:10481000DE2B0E2E0895A0E0F3FCA1E0E0E00E9464
:10482000C52B0E22A22FE3E60895E0913403F09108
:1048300035030895F297ADE7B0E00E94182C0F0100
:104840000895F0E0DE015796AE0FBF1FEC91F0E047
:10485000D0010E94502C9CDFA0DFA93CE0E0BE0705
:104860000895F0E0DE015B96AE0FBF1FEC91F0E023
:1048700094DF0E94182CDF01E4E6F0E00E94502C47
:1048800087CFE02FF0E0DE015396AE0FBF1F0895F3
:10489000A0917603B091770380917803909179038A
:1048A0000895E8EEF3E060E070E00E948D2CDF01F7
:1048B000CB01BBDF662777270895EC91F0E00E94DB
:1048C000BB2BA8E0BCE481E090E00E948D2CE0CFFF
:1048D000E0937603F0937703609378037093790302
:1048E0000895D6DFDECF0E948A2BE5E0F0E060E09D
:1048F00070E00E94102C08950E948A2BE4E1F0E001
:1049000060E070E00E94082C08950E948A2BA43178
:10491000E0E0BE07E0E08E07E0E09E070895E0914A
:104920007E03F0917F036091800370918103A0E585
:10493000B4E180E090E00E944B2CCACFE8EEF3E0B7
:1049400060E070E00895A62DEAE00E94DE2B0E2EB6
:104950000895A22FE3E60E94DE2B0895A0E0F0FC6C
:10496000A1E0E0E00E94C52B0895A0E022FCA1E0B8
:10497000E0E00E94C52BE0210895A0912C0343CED6
:10498000E0912B0345DEFF27662777270895E0E0B7
:104990000E94C52BE0210895EB85FC85A091820340
:1049A000B0918303809184039091850366277727D4
:1049B0000E94082C0E2EEAE0F0E060E070E00E9419
:1049C000102C0895E0936403F09365030895C9DE05
:1049D000AB85BC85882799270E948A2B0895A6302D
:1049E000E0E0BE07E0E08E07E0E09E070895A091BA
:1049F0006403B09165030895E0916403F091650349
:104A00000895EB85FC85A0918203B091830380918A
:104A1000840390918503662777270895E32FA0915B
:104A2000C603B091C7038091C8039091C903FF27C3
:104A3000662777270E943C2A0895AFDEEAE00E94AD
:104A4000402C0895E32FF0E0A091C603B091C70376
:104A50008091C8039091C9030E94BB2B0E943C2AFD
:104A60000DCDA0916603B091670308950E94C02BFD
:104A70000E94ED2C03CDA32FBB27E091C603F0913C
:104A8000C7036091C8037091C903F0CFE09166033A
:104A9000F091670308950E94BB2B0E943C2A089561
:104AA000EAE0F0E00E94632C73CEE0911303B0DDE6
:104AB000FF27662777270895E0936E03F0936F032F
:104AC0000895E0911303F0E0A3DD0E94BB2B0E9448
:104AD0008A2B08950E94462CA0916E03B0916F031B
:104AE0000895E0916E03F0916F030895A091130370
:104AF000BB27E0917E03F0917F036091800370916A
:104B000081030E94C02B0E948A2B0895A0E0F09997
:104B1000A1E0E1E00E94C52B84CD0E22A22FE3E6A6
:104B20000E94C52BE02108950E2EA0911D03ECE3F9
:104B30000E94DE2B0E2208950E94192DA1E0B0E004
:104B40000C94C629E091B203F091B3036091B403D1
:104B50007091B503A2E3B0E00E94052AEDCFAAE36D
:104B6000B0E00E94052AE8CF8EDCACE3B0E0E4CFF1
:104B70000E94212DA1E0B0E00C94C629EAE00E9439
:104B8000E32B0E2E0895AB2DEAE00E94DE2B0E2EB5
:104B9000A0E027FCA1E0E0E00E94C52B0E220895D2
:104BA000A0E0F2FCA1E0E0E00E94C52B0895A92D51
:104BB000EAE00E94DE2B0E2E0895E0E00E94C52B55
:104BC0000E220895E0910E03F0E0E75FFC4F089598
:104BD000E0914403F09145030895E0913103EF5FC4
:104BE000E0933103E0913003A0913103EA17089577
:104BF0000E94DE2B0E2EA0E023FCA1E00895A091E0
:104C00004403B09145030895A0915803B09159030E
:104C10000895E1E00E94F92CEA1B0E944C2D0895B2
:104C2000A091C603B091C7038091C8039091C903B6
:104C30000895E091C603F091C7036091C803709195
:104C4000C9030895A0E0B0E080E09FE30E94762AC7
:104C50000895E093B603F093B7036093B80370939D
:104C6000B9030895E6DFA0E7B3E041CCE2DFA2E7B5
:104C7000B3E03DCCE0919603F091970360919803E7
:104C8000709199030895EAE0F0E00E94502C089595
:104C9000A0919603B0919703809198039091990306
:104CA0000895D0DBD8CBE0939203F0939303609305
:104CB0009403709395030895F0E0EA0FFB1FE093CF
:104CC0004203F0934303AEE30C94A4210E94A42179
:104CD000A0E00C94A421E0914303AE2F0E94A421F4
:104CE000A09142030C94A421B0E0E2E0F0E00E9425
:104CF000632C0895EAE0EEAFEFAFDE01A05CBF4F9A
:104D0000EC930895DE01AF5BBF4FEC930895DE0195
:104D1000AE5BBF4FEC930895DE01AD5BBF4FEC93EC
:104D20000895DE01AC5BBF4FEC930895E9E0ECA37E
:104D3000E0912D03E170EE0FE058AE2FE0912D03CE
:104D4000E695E695E170EE0FEE0FEA0F0E2EA0E06D
:104D5000F199A1E0EA2FEE0FEE0FEE0F0895ECA30C
:104D6000E0912D03E170EE0FE058AE2FE0912D039E
:104D7000E695E695E170EE0FEE0FEA0F0E2EA0E03D
:104D8000F199A1E0EA2FEE0FEE0FEE0FE00DEBA38D
:104D90000895E295E07FEE0FEE0F0895E0E020FC2D
:104DA000E1E0E0930103A0918603B0918703809135
:104DB0008803909189030895A0918603B091870399
:104DC00080918803909189030895AA30E0E0BE079E
:104DD000E0E08E07E0E09E0708951ADCEAE0F0E0EC
:104DE00060E070E008950E948D2CDF01CB01EAE0C5
:104DF000F0E060E070E00E94A72C0895E09170035D
:104E0000F09171030E948F2BE0937203F093730370
:104E10000895A0917203B09173030895FADFEAE058
:104E2000F0E008950E94632CDF01EAE0F0E00E94C8
:104E3000952C0895E4E6F0E060E070E00895BCDFB2
:104E4000EAE0F0E060E070E00895A436E0E0BE073C
:104E5000E0E08E07E0E09E070895A0E020FCA1E0DE
:104E6000EA2FE295E07FABA1EA0FEBA30895A091B2
:104E70003C03B0913D030895FE01F6963D96BF01B7
:104E8000F6CFE8EEF3E00E94502CDF01EAE0F0E01C
:104E90000E94922CDB01EC930895FE01F6963E965B
:104EA000BF01E5CFE4E6F0E00E94502CDF01EAE02C
:104EB000F0E00E94922CDB01EC930895FE01F6963F
:104EC0003F96BF01D4CFDF01EAE0F0E00E94922CD0
:104ED000DB01EC9308950E94922CDB01EC93089582
:104EE000BB27EAE0F0E00E94952C0895FE01F696BB
:104EF0003A96BF010895EAE0F0E094CFDB01EC932D
:104F0000FE01F69608950E94682CDF01CB01EAE0CD
:104F1000F0E060E070E00E94A32C0895A031E7E289
:104F2000BE07E0E08E07E0E09E070895A83EE3E0BC
:104F3000BE07E0E08E07E0E09E07089552DBEAE05E
:104F4000F0E060E070E00895EFAFE4E7DE01A05C20
:104F5000BF4FEC930895DF01CB01E0E0F0E060E1AA
:104F600071EC0E94592B0895DF01CB01E0E0F0E0E5
:104F700066EC72EC0E94592B0895DF01CB01CCCA7C
:104F8000A0918A03B0918B0380918C0390918D0343
:104F9000089550DF28CFF4DFEAE0F0E060E070E051
:104FA0000895ECA1E058ECA3EEE3CECFE0916C03C2
:104FB000F0916D030E948F2BE0936C03F0936D03CF
:104FC000089540DAA4E6B0E080E090E081CAA091C4
:104FD0006C03B0916D030895FE01F6963B96BF01F8
:104FE0000895F5DFE0E1F7E21DCFFE01F6963C966D
:104FF000BF010895ECDFE8EEF3E014CFFE01F69672
:105000003D96BF010895E3DFE4E6F0E00BCFFE013B
:10501000F6963E96BF010895FE01F6963F96BF01B3
:10502000D6DFEAE0F0E00E94952CDB01EC930895D6
:10503000A0917403B09175030895FADFE4E6F0E0FF
:10504000F1CE3F96BF01F4DFEAE0F0E00E94952C3C
:10505000DB01EC930895DE01A05CBF4FEC93089553
:10506000EAE0F0E00E94952C0895E985FA85F6952E
:10507000E79508950E94502C26CFDF01EAE0F0E08A
:105080000E94922C0895A0914803B091490308957D
:10509000EAE0F0E00E94922C0895EAE0F0E01BCFF5
:1050A000ECA1E058ECA3E2E0EEAFEEE34DCFE9E394
:1050B000D2DFE8E327CEE52FF0E0DE01D696AE0F93
:1050C000BF1F08950E94C52B0E2EAE8108950E9429
:1050D000C52B0E2AAE810895AD85BE85D4CDAE8197
:1050E000E5E0F0CFE3E10E94C52BE0290895E72D2C
:1050F000F0E0DE015396AE0FBF1F0895A0917A0332
:10510000B0917B0380917C0390917D030895EC9195
:10511000F0E00E94BB2BA8E0BCE481E090E00E949C
:105120008D2CECCFE0937A03F0937B0360937C03A8
:1051300070937D030895E2DFB4CBEF85F88968DAD8
:10514000662777270E944B2CEDCFA0918203B09168
:10515000830380918403909185030895EBAFF5DF7D
:10516000EAE0F0E060E070E03ECEECAFEEDFEAE0D7
:10517000F0E060E070E00E94A72CEDAF089555DBF1
:10518000F695E79505CBEAA308DBA436E0E0BE0779
:10519000089503DBE4E6F0E00E94502C6ECFFDDAC8
:1051A00072CDFBDA75CFA0915603B09157030895E5
:1051B000E4E6F0E00E94502C60CFE9E3EFAFE0E5D9
:1051C0004ADFEEE39FCDA0914003B09141030895E3
:1051D000A0914C03B0914D030895A0913603B09176
:1051E00037030895E170E795E0E0E795AE2F089565
:1051F000E295EF70E695E170CCDDEA2BAE2F0895D5
:10520000E295EF70E695E695E170E295E07FEE0FAE
:10521000EA2BAE2F0895E295E170E295E07FEA2B4C
:10522000AE2F0895E170EE0FEE0FEE0FEA2BAE2FCA
:105230000895E695E170EE0FEE0FEA2BAE2F08957C
:10524000E695E695E170EE0FEA2BAE2F0895E69510
:10525000E695E695E170EA2B0895FE01ED5BFF4FC0
:10526000E0810895E695E17094DDEA2BAE2F089574
:10527000E695E695E170E295E07FEE0FEA2BAE2F22
:105280000895E695E695E695E170E295E07FEA2BD4
:10529000AE2FECA10895E695E695E695C3CFE2958D
:1052A000EF70E695E170EE0FEE0FEA2BAE2F08954A
:1052B000E295EF70E695E695E170EE0FEA2BAE2FE2
:1052C0000895FE01EE5BFF4FE0810895FE01EC5B67
:1052D000FF4FE0810895E295EF70E69583CFFE01E0
:1052E000EF5BFF4FE0810895E295EF70E695E6955C
:1052F0000895FE01E05CFF4FE0810895FE01EB5B45
:10530000FF4FE0810895E170E295E07FEA2B089578
:10531000E170EE0FEE0FEA2BAE2F0895E17039DD4C
:10532000EA2BAE2F0895E695E170E295E07FEE0F4F
:10533000EA2BAE2F0895E695E695EACFE170EE0FE1
:10534000EA2BAE2F0895E295EF70E695DCCF289812
:1053500085E28A95F1F751E008955E9885E28A9595
:10536000F1F7ECE0E51B089585E28A95F1F75E9A86
:1053700085E28A95F1F708955D9A85E28A95F1F7BD
:10538000289A84E191E00197F1F7E1CF109639F086
:105390008DEC9AE00197F1F7A8951197C9F7089558
:1053A00030976040704009F070580895552342F4DA
:1053B000503811F4E0FF04C03196691F791F6BF07B
:1053C00050E8572711F45F93CFC05F3F31F0660F6D
:1053D000000C57956795752F08955F9300200AF08C
:1053E000CFC0C8C050E8192E1522880F991F9527E5
:1053F000550F879550E8072E0522660F771F7527F2
:10540000550F67950895689401C0E8945F93F2DFA3
:10541000703818F07F3F08F4A7C056E1571BAAF474
:10542000519558300EF4593030F0EFEFFFEF6FEF39
:105430007FE777F91AC077275523B9F0EE0FFF1FE2
:10544000661F771F5A95D1F710C07727583028F07C
:10545000EF2FF62F672F5850F9CF552331F076955F
:105460006795F795E7955A95D1F700200AF45BD137
:105470005F910895689401C0E8943097604070404F
:10548000B1F0002426F0772312F400944CD1172EAB
:105490007EE1112032F07A95EE0FFF1F661F111C7E
:1054A000F9CFEF2FF62F612D5F938ADF5F9108957B
:1054B0004F93AF01FD01DA01AB01BC01CA01402DE0
:1054C000012C142E4F910895EA0FFB1F681F0895B9
:1054D000E095F0956095EF5FFF4F6F4F08955F93F4
:1054E00081DF903871F150E8152604C05F937ADFB0
:1054F000903839F1703821F1572F591B2BF112F4E4
:10550000D7DFFACF583118F0AA27BB2788275830A1
:1055100028F0AB2FB82F88275850F9CF552329F002
:105520008695B795A7955A95D9F7502D512572F0C4
:10553000CBDF38F46795F795E795739513F420C0A2
:10554000B7DF3EDF5F910895D8F7FBCFEA1BFB0B77
:10555000680B51F010F40094BBDF662392F3EE0F5A
:10556000FF1F661F7A95CBF7EE27FF276627772761
:105570005F910895EFEFFFEF6FE77FEF5F91089581
:10558000EFEFFFEF6FE77FE75F9108955F932ADF0B
:10559000703851F3903841F301240894791F23F4B3
:1055A0001CF300203AF3ECCF0F921F932F933F93FD
:1055B0004F93112722279927689FA0018F9F302D95
:1055C000410D591F6B9F300D411D591F8E9F27D0D4
:1055D000BF9F25D06A9F23D0BE9F1DD0AF9F1BD0F9
:1055E000AE9F110D291F391F491F591FE32FF42F9B
:1055F000652F522F4F913F912F911F910F9066234E
:105600002AF0550FEE1FFF1F661F02C073954BF265
:10561000CDDE5F910895100D211D391F02C0200DB0
:10562000311D491F591F08955F93DCDE703821F446
:1056300011200AF49FCFA4CF903809F495CF01240C
:105640000894970B1BF4D4F30020F3CF792F1F930A
:105650002F933F934F931124112722273327442759
:10566000552790E2AE17BF078607410730F0AE1B03
:10567000BF0B860B410B089401C08894551F221F55
:10568000331F111CAA1FBB1F881F441F9A9551F777
:10569000F901612D4F913F912F911F91662332F0B7
:1056A000550FEE1FFF1F661F7A9543F27FDE5F9155
:1056B000089599239AF0772342F0971748F029F438
:1056C000AE17BF07860720F031F0989488940895AC
:1056D0009894089408951894889408957723C2F7AD
:1056E000971798F3A9F7EA17FB07680788F399F368
:1056F000ECCFDFDFE1E009F008F0EE270895D9DF15
:10570000E1E009F008F4EE270895EA0FFB1F681F97
:10571000791F0895AE1BBF0B860B970B0895F1956B
:10572000E195F0400895F09560957095E195FF4FF3
:105730006F4F7F4F0895EE230E2EEA2F19F0E69556
:105740000A94E9F70895EE230E2EFD0121F0F69557
:10575000E7950A94E1F70895F695E795F695E795AC
:10576000F695E795F695E7950895FE2FFF0FFF0B49
:105770006F2F7F2F08956F2F660F660B762F08957A
:105780008B2F880F880B982F0895EA17E1E009F016
:10579000EE270895EA17E1E009F4EE270895AE1721
:1057A000E1E00CF4EE270895AE17E1E00CF0EE27EF
:1057B0000895EA17E1E00CF0EE270895AE17E1E056
:1057C00008F0EE270895EA17E1E008F0EE270895C3
:1057D000EA17FB07E1E009F0EE270895AE17BF07CF
:1057E000E1E008F4EE270895AE17BF07E1E008F006
:1057F000EE270895EA17FB07E1E008F0EE27089589
:10580000EA17FB0768077907E1E009F0EE2708953A
:10581000AE17BF0786079707E1E00CF0EE27089563
:10582000EA17FB0768077907E1E00CF0EE27089517
:10583000FA9FF02DEB9FF00DEA9FE02DF10D0895FA
:105840007A9F702D6B9F700DF89F700DE99F700D02
:105850006A9F602D710DFB9F600D711DE89F600DAB
:10586000711D8827FA9FF02D610D781FEB9FF00DB9
:10587000611D781FEA9FE02DF10D681F781F0895C4
:105880006E2F6A9FF0016B9FF00D089574D0D0DFEA
:105890000EF445DF08957DD0D3DF0EF444DF089584
:1058A0000024112490E1AA0FBB1F001C111C0E1A2A
:1058B0001F0A18F40E0E1F1E01C0A1609A9599F7D9
:1058C000FD01D001089557D0EBDF0EF428DF0895D5
:1058D0003F934F935F93002411244427552730E2D0
:1058E000AA0FBB1F881F991F001C111C441F551FA6
:1058F0000E1A1F0A460B570B28F40E0E1F1E461FCA
:10590000571F01C0A1603A9559F7FD01BC01D001B4
:10591000CA015F914F913F9108953BD0D9DF0EF4BA
:1059200002DF0895BDDFFD010895E894B7FF04C0CC
:10593000A095B09511966894F7FDF1DEB1DFFD01F9
:105940000EF4EDDE0895C4DFFD01BC010895E89476
:1059500097FF09C0A095B09580959095AF5FBF4F18
:105960008F4F9F4F689477FDDEDEB2DFFD01BC01F3
:105970000EF4D9DE0895E894F7FF02C0D0DE6894F3
:10598000B7FF06C0A095B095119600F8039400FAF1
:105990000895E89477FF02C0C6DE689497FF0BC0B5
:1059A0000024A095B095809590951196801D901D2E
:1059B00000F8039400FA0895ED93FD936D937C93A2
:1059C0000895A881B9818A819B810895E883F9832C
:1059D0006A837B830895689401C0E89401D04DDD0B
:1059E000182E862F612D192E972F712D1B2EBF2F4C
:1059F000F12D1A2EAE2FE12D0895129602D0BF017F
:105A00001297119602D0FE2F1197F999FECFFF93AE
:105A1000FFB7F894A1BDB2BDF89AE0B5FFBFFF9102
:105A2000089507D012960F01FB0103D0F0011297E1
:105A3000089507D01196EF93EF2F03D0EF911197B0
:105A40000895F99B02C0A895FCCF9FB7F894A1BD1B
:105A5000B2BDF89A80B5E81719F0E0BDFA9AF99A44
:105A60009FBF089500240E160F0606060706089528
:105A700000240A160B06089500240A160B060806D1
:105A800009060895EA17FB07680779070895AE1716
:105A9000BF07860797070895E894EE2309F06894F6
:105AA0000895AC0FBD1F05900D928A95E1F70895FA
:00000001FF
